:10800000FEDF07EA000000000000000000000000A2
:108010000000000000000000000000000000000060
:108020000000000000000000000000000000000050
:108030000000000000000000000000000000000040
:108040000000000000000000000000000000000030
:02000004001FDB
:020000040020DA
:1000000002D3A0E3A60000EBFEFFFFEA001080E5AC
:100010001EFF2FE1B010C0E11EFF2FE10010C0E570
:100020001EFF2FE1000090E51EFF2FE10E00A0E172
:100030001EFF2FE110FF2FE11EFF2FE108402DE9E9
:1000400008009FE5F6FFFFEB0840BDE81EFF2FE12B
:100050005450212008402DE91C009FE5F0FFFFEBE4
:10006000010010E3FBFFFF0A10009FE5ECFFFFEB30
:100070000840BDE8FF0000E21EFF2FE154502120A0
:100080004050212008402DE90C009FE5E4FFFFEBE4
:100090000840BDE8010000E21EFF2FE1545021207E
:1000A00010402DE90040A0E11C009FE5DCFFFFEBC4
:1000B000200010E3FBFFFF0A0410A0E10C009FE505
:1000C000D1FFFFEB1040BDE81EFF2FE1545021206F
:1000D0004050212008402DE910009FE5D0FFFFEBA4
:1000E000010C10E3FBFFFF1A0840BDE81EFF2FE1E3
:1000F0005450212038402DE90050A0E12040A0E3D9
:10010000044044E23534A0E10F3003E2090053E338
:100110003700838230008392E0FFFFEB000054E35E
:10012000F6FFFF1A2000A0E33840BDE8DBFFFFEA3E
:1001300008402DE9EEFFFFEB0D00A0E3D7FFFFEB3A
:100140000A00A0E30840BDE8D4FFFFEA10402DE913
:10015000D8009FE50110A0E3ABFFFFEBD0009FE5C7
:100160000010A0E3A8FFFFEBC8009FE50010A0E38C
:10017000A5FFFFEBC0009FE50310A0E3A2FFFFEB8C
:10018000B8009FE50010A0E39FFFFFEBA0009FE5F4
:100190000010A0E39CFFFFEBA4009FE5C610A0E3C6
:1001A00099FFFFEB9C109FE59C009FE596FFFFEBFE
:1001B00098009FE59AFFFFEB3F1AC0E3121A81E314
:1001C00088009FE590FFFFEB84009FE50010A0E30F
:1001D0008DFFFFEB0040A0E30400A0E1014084E2BA
:1001E00094FFFFEB960054E3FAFFFF1A64009FE5CB
:1001F0000319A0E384FFFFEB0040A0E30400A0E1AB
:10020000014084E28BFFFFEB960054E3FAFFFF1AF4
:1002100040009FE50010A0E37BFFFFEB14009FE58B
:100220000310A0E378FFFFEB1040BDE81EFF2FE1B5
:100230000450212044502120605021204C50212086
:1002400050502120485021200E01000068502120EC
:1002500004002020940020209800202010402DE948
:100260001C409FE5F918A0E30400A0E166FFFFEB46
:100270000400A0E10C109FE563FFFFEB1040BDE818
:100280001EFF2FE108B400200002F90008402DE90C
:1002900008009FE562FFFFEB0840BDE81EFF2FE16D
:1002A00020B40020F0472DE9A7FFFFEB38029FE5BF
:1002B0009EFFFFEB5CFFFFEB9CFFFFEB0209A0E35F
:1002C0009AFFFFEBE4FFFFEB20A29FE520929FE562
:1002D0001500A0E371FFFFEBEBFFFFEB0040A0E197
:1002E000020000EA66FFFFEB000050E30A00001A7C
:1002F000E5FFFFEB000064E00A0050E1F8FFFF9A21
:100300001500A0E365FFFFEB5DFFFFEB3D4884E2D6
:10031000000050E3094C84E2F4FFFF0A0289A0E3E5
:100320000060A0E3C040A0E30170A0E348FFFFEB42
:10033000C00054E30050A0E12600000A5E00009ACD
:10034000C10054E35700000AC20054E34F00001AF2
:10035000FF3067E2000053E14900000A1800A0E303
:100360004EFFFFEB1800A0E34CFFFFEB1800A0E3EB
:100370004AFFFFEB1800A0E348FFFFEB1800A0E3E3
:1003800046FFFFEBC0FFFFEB0040A0E1BEFFFFEB2D
:10039000000064E0090050E1FBFFFF9A0D00A0E3BC
:1003A0003EFFFFEB0A00A0E33CFFFFEB0A00A0E3E7
:1003B0003AFFFFEB3C019FE55CFFFFEB44FFFFEBE7
:1003C000000000EA22FFFFEB2DFFFFEB000050E3EF
:1003D000FBFFFF1ABDFFFFEA010050E32500000A02
:1003E000040050E3DCFFFF1A0600A0E32BFFFFEB45
:1003F000A5FFFFEBF8409FE50050A0E1A2FFFFEB57
:10040000000065E0040050E1FBFFFF9A0D00A0E34F
:1004100022FFFFEB0A00A0E320FFFFEB0A00A0E3AE
:100420001EFFFFEBD0009FE540FFFFEB08FFFFEB57
:100430002000C0E3470050E3FBFFFF1A0D00A0E3DC
:1004400016FFFFEB2D00A0E314FFFFEB2D00A0E350
:1004500012FFFFEB0D00A0E310FFFFEB0A00A0E38B
:100460000EFFFFEB0A00A0E30CFFFFEB0209A0E385
:10047000EFFEFFEBECFFFFEAC140A0E30560A0E167
:10048000A9FFFFEA065080E00040A0E3FAFFFFEA80
:100490000450C8E7014084E2FF0054E3056086E0B1
:1004A000A1FFFF1AACFFFFEA070050E1AAFFFF1A05
:1004B000075086E0C240A0E3EFFFFFEA800054E36C
:1004C000F2FFFF1AFF6006E2060050E1A2FFFF1AEA
:1004D0000600A0E3017087E2F0FEFFEB808088E277
:1004E000FF7007E2C040A0E3E3FFFFEA7856341252
:1004F000FF083D007F841E00ADDBBA00DADADADAED
:040000030000800079
:00000001FF
